:020000040000FA
:0400000083016328ED
:08000800CF00030E83018C0000
:100010000A088D0004088E008A0183120E089800D9
:100020000F08990010089A0011089B0012089C0004
:1000300013089D0014089E0015089F001608A000D4
:100040001708A1008B18B72B18088E0019088F000D
:100050001A0890001B0891001C0892001D089300CC
:100060001E0894001F08950020089600210897009C
:100070000E0884000D088A000C0E8300CF0E4F0E70
:10008000090083121008130203184B2803194B2888
:1000900001309300003493010034831210081302DE
:1000A000031C57280319572801309300003493018B
:1000B0000034831210081302031D612801309300DD
:1000C00000349301003483128316DD308100640014
:1000D000DD308100831210308316850007308600E2
:1000E0008312A601A701A801A201A301A401AD01E9
:1000F000AE01A501051085100511861306138612A1
:10010000061286110130A9008B17831601170B16F2
:10011000831683122508950001309300150890007E
:1001200059208312013093061308131C982888283D
:100130008312640083120030061C9F280130831252
:10014000A2000030861CA52801308312A3000030D5
:10015000061DAB2801308312A4002208950001304F
:10016000930015089000592083121308131CB92816
:10017000A60A831223089500013093001508900009
:10018000592083121308131CC628A70A83122408B7
:100190009500013093001508900059208312130830
:1001A000131CD328A80A8312250895000130930058
:1001B00015089000592083121308131CE0289A2870
:1001C00083122908950001309300150890005920EA
:1001D00083121308131C4B2926089500183093002E
:1001E00015089000412083121308950026089600F8
:1001F0001E309300160890004D2083121308150836
:100200009305131C06292608AA00092983121B300E
:10021000AA00831227089500183093001508900053
:100220004120831213089500270896001E30930082
:10023000160890004D208312130815089305131C0F
:1002400024292708AB00272983121B30AB00831217
:10025000280895001830930015089000412083125B
:1002600013089500280896001E3093001608900089
:100270004D208312130815089305131C42292808E2
:10028000AC00452983121B30AC008312A901A601E2
:10029000A701A801882883128B13AF01B001B10117
:1002A000B201B301B4012B08950016301507950073
:1002B0002708930015089000412083121308950029
:1002C000270896002B08970004301707930016089C
:1002D000900041208312130815089305131C7229FE
:1002E0000130B00083122B089500043015079500EB
:1002F00027089300150890004D20831201309306C3
:1003000013089500270896002B0897000430170261
:100310009300160890004D208312013093061308B5
:1003200015089305131C96290130B30083122B087E
:1003300095001630150295002708930015089000C7
:100340004D20831213089500270896002B0897006C
:10035000043017029300160890004D2083121308F2
:1003600015089305131CB6290130AF0083122A0823
:100370009500163015079500260893001508900083
:100380004120831213089500260896002A0897003A
:1003900004301707930016089000412083121308B9
:1003A00015089305131CD6290130B10083122A08C1
:1003B0009500043015079500260893001508900055
:1003C0004D208312013093061308950026089600ED
:1003D0002A089700043017029300160890004D2059
:1003E000831201309306130815089305131CFA298C
:1003F0000130B40083122A089500163015029500CA
:1004000026089300150890004D20831213089500CC
:10041000260896002A089700043017029300160851
:1004200090004D208312130815089305131C1A2AF7
:100430000130B20083122C08950016301507950084
:100440002808930015089000412083121308950096
:10045000280896002C089700043017079300160808
:10046000900041208312130815089305131C392AA4
:10047000051483122C0895000430150795002808F0
:100480009300150890004120831213089500280856
:1004900096002C089700043017029300160890006D
:1004A00041208312130815089305131C592A0510BF
:1004B000851083122C089500163015029500280827
:1004C0009300150890004D2083121308950028080A
:1004D00096002C089700043017029300160890002D
:1004E0004D208312130815089305131C782A8514D0
:1004F00083122808950005309300150890004D20C0
:1005000083121308950028089600283093001608D7
:10051000900041208312130815089304131C922A9B
:1005200005108510831226089500053093001508E4
:1005300090004D208312130895002708960005307F
:100540009300160890004D20831213081508930499
:10055000131CAF2A8611061286120613AC2B8312C7
:10056000340895000130930015089000592083123B
:100570001308950033089600013093001608900088
:1005800059208312130815089305131CCB2A8611D2
:1005900006128612061383122F089500013093006D
:1005A000150890005920831213089500340896000E
:1005B0000130930016089000592083121308150883
:1005C0009305131CE72A0612061386168615831256
:1005D00030089500013093001508900059208312CF
:1005E0001308950034089600013093001608900017
:1005F00059208312130815089305131C032B861129
:1006000086120616061783123108950001309300F2
:10061000150890005920831213089500330896009E
:100620000130930016089000592083121308150812
:100630009305131C1F2B06128612861506178312AC
:10064000320895000130930015089000592083125C
:1006500013089500330896000130930016089000A7
:1006600059208312130815089305131C3B2B861180
:100670000613061686168312320895000130930081
:100680001508900059208312130895002F08960032
:1006900001309300160890005920831213081508A2
:1006A0009305131C572B8611061206138616831208
:1006B0002F089500013093001508900059208312EF
:1006C0001308950031089600013093001608900039
:1006D00059208312130815089305131C732B061257
:1006E0008612061386158312320895000130930096
:1006F00015089000592083121308950030089600C1
:100700000130930016089000592083121308150831
:100710009305131C8F2B861106128612061783125F
:10072000310895000130930015089000592083127C
:1007300013089500300896000130930016089000C9
:1007400059208312130815089305131CAB2B86112F
:1007500086120613061683128312A501A601A701AD
:10076000A801A201A301A4018B178828CB2B831217
:100770002508950000309300150890005920831239
:100780001308131CC62B0130A500C82B8312A5012A
:0807900083128B102428831250
:02400E00FE3F73
:00000001FF
